BL51 BANKED LINKER/LOCATER V6.00                                                        09/05/2017  17:40:44  PAGE 1


BL51 BANKED LINKER/LOCATER V6.00, INVOKED BY:
C:\KEIL_UV3\C51\BIN\BL51.EXE main.obj TO MA82G5Dxx RAMSIZE (256)


MEMORY MODEL: SMALL


INPUT MODULES INCLUDED:
  main.obj (MAIN)
  C:\KEIL_UV3\C51\LIB\C51S.LIB (?C_STARTUP)


LINK MAP OF MODULE:  MA82G5Dxx (MAIN)


            TYPE    BASE      LENGTH    RELOCATION   SEGMENT NAME
            -----------------------------------------------------

            * * * * * * *   D A T A   M E M O R Y   * * * * * * *
            REG     0000H     0008H     ABSOLUTE     "REG BANK 0"
            DATA    0008H     0004H     UNIT         ?DT?MAIN
            DATA    000CH     0001H     UNIT         _DATA_GROUP_
            IDATA   000DH     0001H     UNIT         ?STACK

            * * * * * * *   C O D E   M E M O R Y   * * * * * * *
            CODE    0000H     0003H     ABSOLUTE     
            CODE    0003H     004AH     UNIT         ?PR?MAIN?MAIN
            CODE    004DH     0019H     UNIT         ?PR?_IAP_READ?MAIN
            CODE    0066H     0016H     UNIT         ?PR?_PAGEP_WRITE?MAIN
            CODE    007CH     0016H     UNIT         ?PR?_PAGEP_READ?MAIN
            CODE    0092H     0016H     UNIT         ?PR?_IAP_PROGRAM?MAIN
            CODE    00A8H     0014H     UNIT         ?PR?_IAP_ERASE?MAIN
            CODE    00BCH     000CH     UNIT         ?C_C51STARTUP



OVERLAY MAP OF MODULE:   MA82G5Dxx (MAIN)


SEGMENT                          DATA_GROUP 
  +--> CALLED SEGMENT          START    LENGTH
----------------------------------------------
?C_C51STARTUP                  -----    -----
  +--> ?PR?MAIN?MAIN

?PR?MAIN?MAIN                  000CH    0001H
  +--> ?PR?_PAGEP_READ?MAIN
  +--> ?PR?_PAGEP_WRITE?MAIN
  +--> ?PR?_IAP_ERASE?MAIN
  +--> ?PR?_IAP_PROGRAM?MAIN
  +--> ?PR?_IAP_READ?MAIN



SYMBOL TABLE OF MODULE:  MA82G5Dxx (MAIN)

  VALUE           TYPE          NAME
  ----------------------------------
BL51 BANKED LINKER/LOCATER V6.00                                                      09/05/2017  17:40:44  PAGE 2



  -------         MODULE        MAIN
  C:0000H         SYMBOL        _ICE_DUMMY_
  D:0090H         PUBLIC        P1
  D:00A0H         PUBLIC        P2
  D:00E7H         PUBLIC        ISPCR
  D:00C0H         PUBLIC        XICON
  D:00B0H         PUBLIC        P3
  D:00E8H         PUBLIC        P4
  D:00F8H         PUBLIC        P6
  C:00A8H         PUBLIC        _IAP_Erase
  C:007CH         PUBLIC        _PageP_Read
  D:00A8H         PUBLIC        IE
  D:0008H         PUBLIC        IAP_Var0
  D:00B8H         PUBLIC        IP0L
  D:0009H         PUBLIC        IAP_Var1
  D:000AH         PUBLIC        IAP_Var2
  C:0050H         PUBLIC        _IAP_Read
  D:000BH         PUBLIC        IAP_Var3
  C:0066H         PUBLIC        _PageP_Write
  D:00BFH         PUBLIC        CKCON1
  D:00D8H         PUBLIC        CCON
  C:0003H         PUBLIC        main
  D:00E6H         PUBLIC        SCMD
  D:00E3H         PUBLIC        IFADRH
  D:00E5H         PUBLIC        IFMT
  D:00E4H         PUBLIC        IFADRL
  D:0088H         PUBLIC        TCON
  D:00E2H         PUBLIC        IFD
  D:0098H         PUBLIC        S0CON
  D:00C8H         PUBLIC        T2CON
  C:0092H         PUBLIC        _IAP_Program
  D:00D0H         PUBLIC        PSW
  -------         PROC          _PAGEP_WRITE
  D:0007H         SYMBOL        Addr
  D:0005H         SYMBOL        Data
  C:0066H         LINE#         16
  C:0066H         LINE#         17
  C:0066H         LINE#         18
  C:0069H         LINE#         19
  C:006BH         LINE#         20
  C:006DH         LINE#         21
  C:0070H         LINE#         22
  C:0073H         LINE#         23
  C:0076H         LINE#         24
  C:0079H         LINE#         25
  C:007BH         LINE#         26
  -------         ENDPROC       _PAGEP_WRITE
  -------         PROC          _PAGEP_READ
  D:0007H         SYMBOL        Addr
  -------         DO            
  D:0007H         SYMBOL        Data
  -------         ENDDO         
  C:007CH         LINE#         28
  C:007CH         LINE#         29
  C:007CH         LINE#         32
  C:007FH         LINE#         33
BL51 BANKED LINKER/LOCATER V6.00                                                      09/05/2017  17:40:44  PAGE 3


  C:0082H         LINE#         34
  C:0084H         LINE#         35
  C:0087H         LINE#         36
  C:008AH         LINE#         37
  C:008DH         LINE#         38
  C:008FH         LINE#         39
  C:0091H         LINE#         41
  C:0091H         LINE#         42
  -------         ENDPROC       _PAGEP_READ
  -------         PROC          _IAP_ERASE
  D:0007H         SYMBOL        AddrH
  D:0005H         SYMBOL        AddrL
  C:00A8H         LINE#         45
  C:00A8H         LINE#         46
  C:00A8H         LINE#         47
  C:00AAH         LINE#         48
  C:00ACH         LINE#         49
  C:00AFH         LINE#         50
  C:00B2H         LINE#         51
  C:00B5H         LINE#         52
  C:00B8H         LINE#         53
  C:00BBH         LINE#         54
  -------         ENDPROC       _IAP_ERASE
  -------         PROC          _IAP_PROGRAM
  D:0007H         SYMBOL        AddrH
  D:0005H         SYMBOL        AddrL
  D:0003H         SYMBOL        Dta
  C:0092H         LINE#         56
  C:0092H         LINE#         57
  C:0092H         LINE#         58
  C:0094H         LINE#         59
  C:0096H         LINE#         60
  C:0098H         LINE#         61
  C:009BH         LINE#         62
  C:009EH         LINE#         63
  C:00A1H         LINE#         64
  C:00A4H         LINE#         65
  C:00A7H         LINE#         66
  -------         ENDPROC       _IAP_PROGRAM
  -------         PROC          L?0009
  -------         ENDPROC       L?0009
  -------         PROC          _IAP_READ
  D:0007H         SYMBOL        AddrH
  D:0005H         SYMBOL        AddrL
  -------         DO            
  D:0007H         SYMBOL        Dta
  -------         ENDDO         
  C:0050H         LINE#         68
  C:0050H         LINE#         69
  C:0050H         LINE#         72
  C:0052H         LINE#         73
  C:0054H         LINE#         74
  C:0057H         LINE#         75
  C:005AH         LINE#         76
  C:005DH         LINE#         77
  C:0060H         LINE#         78
  C:0063H         LINE#         80
BL51 BANKED LINKER/LOCATER V6.00                                                      09/05/2017  17:40:44  PAGE 4


  C:0065H         LINE#         81
  C:0065H         LINE#         82
  -------         ENDPROC       _IAP_READ
  -------         PROC          MAIN
  -------         DO            
  D:000CH         SYMBOL        tmp
  -------         ENDDO         
  C:0003H         LINE#         84
  C:0003H         LINE#         85
  C:0003H         LINE#         87
  C:0006H         LINE#         89
  C:000DH         LINE#         91
  C:0014H         LINE#         93
  C:001BH         LINE#         94
  C:0020H         LINE#         95
  C:0026H         LINE#         96
  C:002CH         LINE#         97
  C:0032H         LINE#         99
  C:0039H         LINE#         100
  C:003EH         LINE#         101
  C:0043H         LINE#         102
  C:004BH         LINE#         104
  -------         ENDPROC       MAIN
  -------         ENDMOD        MAIN

Program Size: data=14.0 xdata=0 code=200
LINK/LOCATE RUN COMPLETE.  0 WARNING(S),  0 ERROR(S)
